:04000000B601D32949
:100008000800B616B61EB612B6190E28B615472041
:10001800031835280830A3005B20A20DA30B102875
:10002800B61E402065206120B61A35203A202208E5
:100038000310CE29B616B61EB61236192828FE3970
:10004800B70036150310CE29361A3028A600361602
:1000580047200318352826084E2003183528B61ED1
:10006800CE294020652036113612B6113A08840090
:1000780038088417800446283A088400380980051F
:100088008417800508003A20652040206120370841
:10009800B6190138A2000830A300A20D03183A20AF
:1000A800031C402065206120A30B51283A206520BD
:1000B8003A08840038080005FF3E3B0884003909E7
:1000C80043283B08840039083D282C08A0002D0847
:1000D800A1000130A20064009520031C8228A20B15
:1000E8006F28FF30A007031CA107031CCE29FA3094
:1000F800A2006F286400952003187E28E720A80135
:100108000830A300E82095200318A80AAB1EA80110
:10011800A20CA30B8628AB1AA213E820031422080A
:1001280008003A08840038088417800484130005FE
:100138002B1B3806FF3E0800A400290803140319E6
:10014800CE29C921031C0800A000251883172408FC
:100158008400200880008313A40AA903A1280408A6
:10016800A6003A088400F030B7050830A70003104D
:100178000318B70ACD20A60CA70BBC280000AB1AA1
:10018800370CCD20D1210314CD202F08A3002E0831
:100198003A298413AB1FDC28000838042B1F3806C3
:1001A8008000841700083804031C38068000E828FB
:1001B80000083804031C38062B1B380680008417F7
:1001C80038098005E82837172B081F39003EA10099
:1001D8002A080E3E0318A10A371F47293713A00023
:1001E80002307E214729B71329080319B7170530AC
:1001F800A8002730A30010300D210330A300E830F9
:100208000D21A30164300D21A3010A300D2124081A
:100218001429A2002508A1002408A000972120087D
:10022800A000A8030319B713290803191E292802D7
:10023800031808002008031DB713B71B0800303E39
:10024800C92901308A002808073982070134023495
:100258000434083410342034403480348317800147
:10026800840AFF3E031D3329CE29A301A200FF30D3
:10027800A207031CA307031CCE290330A100E73003
:1002880047213B29A101FC3EA000A109031C5229DA
:10029800FF300000A00703184D29A0076400A10F34
:1002A8004C290800A8002521A001A101A81DA00033
:1002B800A819A1002008CE29A400A201A301682939
:1002C800A10CA00CA20DA30DFF3E0318642924085D
:1002D80076212208A0042308A1042008080003109E
:1002E800A00DA10DFF3E031873292008CE29031085
:1002F800A10CA00CFF3E03187B292008CE29A301DE
:10030800A20001308729A80023082102031D8E2995
:10031800220820020430031801300319023028058E
:10032800031DFF30CE291030A600A501A401210D20
:10033800A40DA50D2208A4022308031C230FA5025F
:100348000318AD292208A40723080318230FA507BB
:100358000310A00DA10DA60B9B292008CE29103053
:10036800A800A101A001A70CA60C031CC129220802
:10037800A00723080318230FA107A10CA00CA50CA4
:10038800A40CA80BB7292408CE29840031088A00B8
:10039800300882008313031383126400080020309E
:1003A800840060308A013321A030840050308A01F3
:1003B80033211030840060308A013221903084006B
:1003C80060308A013221831607309F009901831219
:1003D8009801831602309800C501C60186100611DF
:1003E8008801071087100711831207118610013042
:1003F8008A013921861464308A0139218A110A1246
:10040800B02E071083162808831288008A110A1252
:10041800122A071483162A088312880087100000FE
:1004280087140710080083164330AA0083128A0134
:100438000D228316FF30880083120714061100006E
:1004480008088316B500831206150710831688015D
:100458008312080083160130B60083128A110A122B
:100468009E2283164630AA0083128A010D2279083B
:100478008316A80083128A01052277088316A8002C
:1004880083128A0105227D08A0007E08A100083099
:10049800A200A3018A0197212408B2002508B3000D
:1004A80032088A015621B2002108B3003208A000A0
:1004B8003308A10008308A0160218316B200831234
:1004C8008A011722640083163608003C8A110A1232
:1004D8008312031D772A831635083204B400831269
:1004E8008A110A127C2A831635083206B400831250
:1004F80083164630AA0083128A010D2279088316D2
:10050800A80083128A01052277088316A80083129F
:100518008A01052283164230AA0083128A010D221D
:1005280083163408A80083128A0105228316B601AF
:1005380083120800831620088312A6008316210858
:100548008312A7002030A200A3018A01B3218316D9
:10055800A600831225088316A70083127D08A00031
:100568007E08A1000830A200A3018A019721831602
:10057800A400831221088316A500260824078312E5
:10058800B200831627080318013E25078312B3001B
:1005980000303207F50010300318013E3307F6002B
:1005A8007608F700F8017508F900FA0108008316C3
:1005B8003E083B078312FD00FE01FE0D83163F082F
:1005C8003C07A000A101A10D83128A0132228316E3
:1005D8003E083B028312FD00FE01031CFE03831646
:1005E8003F083C07A000A101A10D83128A01322215
:1005F80083163B083E078312FD00FE01FE0D83169D
:100608003F083C02A000A101031CA10383128A0138
:10061800322283163E083B028312FD00FE01031CB2
:10062800FE0383163F083C02A000A101031CA1039E
:1006380083128A01322283163F083B078312FD008A
:10064800FE01FE0D83163E083C07A000A101A10D86
:1006580083128A01322283163F083B028312FD006F
:10066800FE01031CFE0383163C083E07A000A101FF
:10067800A10D83128A01322283163B083F07831299
:10068800FD00FE01FE0D83163E083C02A000A101FC
:10069800031CA10383128A01322283163F083B02FE
:1006A8008312FD00FE01031CFE0383163E083C0274
:1006B800A000A101031CA10383128A0132220800B1
:1006C8008316BE013D08BF0003103D0D8312B20022
:1006D800B301B30D3208023C8316A200831233081B
:1006E800031C013E003C8316A3008312640083169A
:1006F8003E083F028A110A128312031CD52B8A0175
:10070800DB2264008A110A1283168310A31F831444
:1007180083128318AD2B0430A600A70183163E0868
:100728008312A200A3018A01B321B2002508B300F5
:100738000630B2070318B30A32088316A2078312D9
:1007480033080318013E8316A30783128A110A127D
:10075800D02B83163F083E028312B200B301031C5C
:10076800B3030430A600A7013208A2003308A3008F
:100778008A01B321B2002508B3000A30B207031872
:10078800B30A32088316A207831233080318013EFE
:100798008316A307BF0383128316BE0A83128A0136
:1007A8007A2B08008316BE013D08BF0003103D0DDB
:1007B8008312B200B301B30D3208023C8316A200C3
:1007C80083123308031C013E003C8316A3008312E6
:1007D800640083163E083F028A110A128312031C22
:1007E800152C8A01DB220430A600A70183163E08D7
:1007F8008312A200A3018A01B321B2002508B30025
:100808000630B2070318B30A32088316A207831208
:1008180033080318013E8316A307BE0A83128A0110
:10082800EC2B08008316BE013D08BF0003103D0DE8
:100838008312B200B301B30D3208023C8316A20042
:1008480083123308031C013E003C8316A300831265
:10085800640083163E083F028A110A128312031CA1
:100868005D2C8A01DB2283163F083E028312B20008
:10087800B301031CB3030430A600A7013208A20089
:100888003308A3008A01B321B2002508B3000A3057
:10089800B2070318B30A32088316A2078312330873
:1008A8000318013E8316A307BF03BE0A83128A01F9
:1008B8002C2C080064008316370838028A110A12A3
:1008C800831203186D2C831637083802B707B8024D
:1008D80083126400831639083A028A110A128312B5
:1008E80003187C2C831639083A02B907BA02831216
:1008F80008008A015E2483163708AD00831264005D
:1009080083162D0838028A110A128312031CA72C99
:1009180083162D088312FD00FE0183163908A000F6
:10092800A10183128A01322283163A08A000A1018C
:1009380083128A01322283164408AD078A110A12EB
:100948008312031C832C83163908AD0083126400BC
:1009580083162D083A028A110A128312031CCD2C21
:1009680083162D08A000A10137088312FD00FE019F
:100978008A013222831638088312FD00FE018A019B
:10098800322283164408AD078A110A128312031C07
:10099800AB2C080083164630AA0083128A010D2268
:1009A8008316A80183128A01052283161030A80035
:1009B80083128A01052283164C30AA0083128A0109
:1009C8000D2283164230AA0083128A010D22831653
:1009D8000130AD0083126400813083162D028A1124
:1009E8000A1283120318182D83160130B0008312DF
:1009F80064002130831630028A110A128312031808
:100A0800112D8316A80183128A0105228316B00AC4
:100A18008A110A128312031DFC2C8316AD0A8A114F
:100A28000A128312031DEF2C080083164630AA0011
:100A380083128A010D228316A80183128A010522D6
:100A480083161030A80083128A0105220800831635
:100A58004630AA0083128A010D228316A801831248
:100A68008A0105228316A80183128A0105228316AA
:100A78004C30AA0083128A010D2283164230AA0044
:100A880083128A010D2283160130AD00831264009F
:100A9800113083162D028A110A1283120318752D3C
:100AA80083160130B00083126400213083163002AF
:100AB8008A110A12831203186E2D83162030A8009B
:100AC80083128A0105228316B00A8A110A12831238
:100AD800031D582D8316AD0A8A110A128312031DAD
:100AE8004B2D83164630AA0083128A010D228316E5
:100AF800A80183128A0105228316A801831208001F
:100B080083164030AA0083128A010D228316AD0194
:100B180083126400083083162D028A110A12831288
:100B28000318BE2D83162D08073C8A110A1283125A
:100B3800031CB52D8A110A12A7258316A800831253
:100B48008A110A12B52D05308A0083162D088312E2
:100B580082073034873407341F3452347F342034CA
:100B680000348A0105228316AD0A8A110A128312FB
:100B7800031D8D2D83164430AA0083128A010D228D
:100B88008316AD0183126400063083162D028A1184
:100B98000A1283120318F62D83162D08053C8A11B4
:100BA8000A128312031CED2D8A110A12E1258316FD
:100BB800A80083128A110A12ED2D05308A008316C7
:100BC8002D0883128207003400347F340034103437
:100BD8007F348A0105228316AD0A8A110A1283120C
:100BE800031DC72D83165A30AA0083128A010D22CD
:100BF8008316A80183128A01052283165B30AA0096
:100C080083128A010D2283160130A80083128A01FB
:100C1800052283165830AA0083128A010D228316F2
:100C28001630A80083128A0105228A01CE248A017F
:100C38002B2583164630AA0083128A010D228316BB
:100C4800A80183128A0105228316A80183128A014A
:100C5800052283164C30AA0083128A010D228316BE
:100C68004230A80083128A0105228316A801831244
:100C78008A01052283165D30AA0083128A010D229B
:100C880083160430A80083128A0105228316863051
:100C9800A80083128A01052283165930AA008312FC
:100CA8008A010D2283161430A80083128A010522B6
:100CB80083164C30AA0083128A010D22080083167D
:100CC8004630AA0083128A010D2275088316A800EF
:100CD80083128A01052276088316A80083128A01E6
:100CE800052283162B08AA0083128A010D22080008
:100CF80083162D083C3E840000088312B200FF30A2
:100D0800A200A20A22080F3C8A110A12031CAF2E65
:100D18008A110A129B2632028A110A12031D852E95
:100D280022088316C00083128A110A12AF2E0630D9
:100D38008A00220882073034313432343334343470
:100D480035343634373438343934613462346334C2
:100D580064346534663408008A0184258316423079
:100D6800AA0083128A010D228316AD018312640042
:100D78003D3083162D028A110A1283120318472F59
:100D880083162D083C3C8A110A128312031C3E2F3D
:100D98008A110A12D5268316A80083128A110A120C
:0E0DA8003E2F07308A0083162D088312002F7D
:100E000082072034503449344334203443346F341F
:100E10006E34743472346F346C346C3465346434CE
:100E2000203453344534443431343334333430345F
:100E300020346F346E342034613420342034203434
:100E4000203420344834793475346E346434613459
:100E5000693420344C34433444342034323435340F
:100E600036347834313432343834203444346934CC
:100E7000733470346C346134793421348A0105223E
:100E80008316AD0A8A110A128312031DBB2E073086
:100E9000A300D0308A013A2183168030BB00403055
:100EA000BC002830BD0083128A0164238A01D62346
:100EB0008A01162483161430BD0083128A0164232C
:100EC00083160230C4004030B700C030B800143080
:100ED000B9006E30BA0083128A017D240B30A30062
:100EE000B8308A013A218A01CE248A012B25C530E7
:100EF000F500F60183164C30AB0083128A0163269D
:100F000083164230AA0083128A010D228316AD0196
:100F100083126400163083162D028A110A1283127E
:100F20000318C82F83162D08153C8A110A12831244
:100F3000031CBF2F8A110A12A3278316A80083124D
:100F40008A110A12BF2F07308A0083162D088312D8
:100F50008207503449344334203443346F346E3480
:100F6000743472346F346C346C34653464342034CB
:100F700053344534443431343334333430348A01D7
:100F800005228316AD0A8A110A128312031D892FC6
:100F9000E330F500F60183164C30AB0083128A0172
:100FA000632683164230AA0083128A010D2283161B
:100FB000AD01831264001B3083162D028A150A12BC
:100FC00083120318252883162D081A3C8A150A1245
:100FD0008312031C1C288A110A12F4278316A80006
:100FE00083128A150A121C2808308A0083162D08DD
:040FF0008312002840
:1010000082075534733469346E3467342034503475
:101010006934633442346134733469346334503432
:1010200072346F3420345634653472342E342034A4
:1010300032342E34333432348A0105228316AD0A19
:101040008A110A128312031DDA2F0530F5000130D0
:10105000F60083164C30AB0083128A016326831698
:101060004230AA0083128A010D228316AD01831239
:101070006400153083162D028A150A128312031894
:10108000762883162D08143C8A150A128312031C35
:101090006D288A150A1252208316A80083128A1519
:1010A0000A126D2808308A0083162D0883128207E1
:1010B000523461346E346A346934743420344434C4
:1010C00069346F346C3420342D34203443344F343D
:1010D0004D3450345334793473348A0105228316E5
:1010E000AD0A8A150A128312031D38282430F50030
:1010F0000130F60083164C30AB0083128A01632660
:1011000083164230AA0083128A010D228316AD0194
:1011100083126400173083162D028A150A12831277
:101120000318C92883162D08163C8A150A12831243
:10113000031CC0288A150A12A3208316A800831254
:101140008A150A12C02808308A0083162D088312D7
:10115000820768347434743470343A342F342F3442
:101160007734773477342E3463346F346D3470349D
:1011700073347934733431342E3463346F346D34D2
:101180008A0105228316AD0A8A150A128312031DED
:101190008928FD01FE017D08A0007E08A100A301B1
:1011A000FF308A0184218A150A12031DEB28831659
:1011B000A001A10183128A01322283167F30A00090
:1011C000A10183128A013222FD0A0319FE0A8A153F
:1011D0000A12031DCB288316A001A10183128316D6
:1011E00020088312A000831621088312A100A30106
:1011F0007F308A0184218A150A12031D1129FD01FD
:10120000FE018A013222FF30FD00FE018A013222F6
:101210008316A00A0319A10A8A150A128312031D54
:10122000EF2883160A30B700F530B8000A30B9004D
:101230007530BA000230C40083128A017D248316FF
:101240005230A000A10183122030FD00FE017D0874
:10125000A0007E08A100A301D4308A0184218A1550
:101260000A12031D3C298A013222FD0A0319FE0AD3
:101270008A150A12031D27298316B001AD01B10199
:1012800083122030FF0083160A30AC008312F50170
:10129000F601FD01FE018316A001A1017830AE0028
:1012A000AF0183120730BA008030B8002030AA00A6
:1012B000AB018A017E202A3C8A150A12031D592996
:1012C0000930A9007E30B000B101A5016B308A0160
:1012D000A0208316AD0183126400093083162D020D
:1012E0008A150A1283120318B42983162D086B3E3F
:1012F000840000088312B200FF30A200A20A220874
:101300000F3C8A150A12031CA8298A150A12942177
:1013100032028A150A12031D7E2922088316C00094
:1013200083128A150A12A82909308A002208820726
:101330003034313432343334343435343634373471
:101340003834393461346234633464346534663437
:1013500083162D086B3E840040088000AD0A8A1574
:101360000A128312031D6C297208A000A101043027
:101370008A017621B2002108B30073083204831673
:10138000AC0083126C08A000A10104308A01762110
:10139000B2002108B3006D083204FF006E08A000FF
:1013A000A10104308A017621B2002108B3006F0840
:1013B0003204F6007008A000A10104308A017621F1
:1013C000B2002108B30071083204F5007508F3007B
:1013D0007608F4006B088316B00064003008003C07
:1013E0008A150A12831203198D2B640083163008A4
:1013F000013C8A150A1283120319B32A640083166A
:101400003008043C8A150A1283120319132A640057
:1014100083163008053C8A150A1283120319212A03
:101420008A150A1252298316E830AE00AF018312E2
:10143000FD01FE018316A001A10183128A150A1283
:10144000A22B8A012B257F038316AE002C03AF004D
:101450008312FD01FE018316A001A10183128A01FE
:10146000192583164230AA0083128A010D22FD013C
:10147000FE017D08A0007E08A10083162E088312BD
:101480008A0183218A150A12031D862A8316A00168
:10149000A1018312831620088312A000831621085D
:1014A0008312A10083162F0883128A0183218A15D3
:1014B0000A12031D7F2A0730BA001030B800073027
:1014C000BB000830B900A0308A01202074088A01CE
:1014D000202073088A0120208A0105208316A80095
:1014E00083128A010522F30A0319F40A8316A00A5B
:1014F0000319A10A8A150A128312031D4A2AFD0A3A
:101500000319FE0A8A150A12031D392A0730BA0088
:101510004030B8002030AA00AB01AE01AF0144302A
:101520008A01B42069308A01B42073308A01B42062
:1015300070308A01B4206C308A01B42061308A0195
:10154000B42079308A01B42065308A01B420643037
:101550008A01B4200A308A01B4200D308A01B420F7
:101560008A150A1252290730BA008030B80020309C
:10157000AA00AB018830AC001330AD008A016920AD
:101580008A150A12031C312C5D3C8A150A12031DB0
:10159000BE2A7F08A9006930B000B101A5013C3026
:1015A0008A01A0208A150A12031C312C8316AD0172
:1015B0008312FF307F07B400FF300318013EB500EF
:1015C00083162D088312A000A1013508A30034085A
:1015D0008A0184218A150A12031D2D2B83162D08DA
:1015E0003C3E840000088312B200FF30A200A20A31
:1015F00022080F3C8A150A12031C212B8A150A1295
:101600000D2332028A150A12031DF72A22088316B7
:10161000C00083128A150A12212B0B308A0022087F
:101620008207303431343234333434343534363460
:101630003734383439346134623463346434653473
:10164000663483162D083C3E840040088000AD0AB5
:101650008A150A128312031DD92A8316AD0183123B
:10166000FF307F07B400FF300318013EB50083163A
:101670002D088312A000A1013508A30034088A01B7
:1016800084218A150A12031D8A2B83162D083C3EDD
:10169000840000088312B2003208A000A1010430C7
:1016A0008A017621B2002108B300013083162D078C
:1016B0008312B400B501B50D34083C3E8400000827
:1016C000B400340832048316A80007308312BA002D
:1016D0001030B8000730BB000830B900A0308A01D4
:1016E000202074088A01202073088A012020831694
:1016F000280883128A011E200A308A013921F30A40
:101700000319F40A02308316AD078A150A128312F0
:10171000031C302B8A150A12B32A8A012B25831643
:10172000F830AE00AF018312FD01FE018316A00167
:10173000A10183128A01192583164230AA0083125F
:101740008A010D220730BA008030B8002030AA008C
:10175000AB01D030AC000730AD008A0169208A159A
:101760000A12031C52295D3C8A150A12031DAD2B77
:101770007F08A9006930B000B101A5013C308A01A1
:10178000A0208A150A12031C52298316AD01831268
:10179000FF307F07B400FF300318013EB500831609
:1017A0002D088312A000A1013508A30034088A0186
:1017B00084218A150A12031DEB2B8A017C268316CD
:1017C0002D083C3E840040088000AD0A8A150A12AC
:1017D0008312031DC82B8316AD018312FF307F07D0
:1017E000B400FF300318013EB50083162D088312A4
:1017F000A000A1013508A30034088A0184218A15BC
:101800000A12031D2E2C83162D083C3E840000086E
:101810008312B2003208A000A10104308A017621AF
:10182000B2002108B300013083162D078312B400E3
:10183000B501B50D34083C3E84000008B4003408FE
:1018400032048316A80083128A010522023083160F
:10185000AD078A150A128312031CEE2B8A150A1291
:10186000A22B0730BA004030B8002030AA00AB01EC
:10187000AE01AF016C308A01B42061308A01B4201E
:1018800073308A01B42074308A01B42020308A0178
:10189000B42062308A01B42079308A01B4207430D7
:1018A0008A01B42065308A01B42020308A01B42036
:1018B00061308A01B42074308A01B4203A308A0140
:1018C000B420A9017308A4007408A500B330B000C7
:1018D000B1018A01F7200A308A01B4200D308A0153
:1018E000B4208A150A12522963008A150A12742C30
:02400E00753DFE
:00000001FF
